:100000000EC0189518951895189518951895189567
:1000100018951895189518951895189518958FEDA9
:100020008DBFC0ECE8EB4E2EDD275D2EEEE7F0E055
:10003000A0E6B0E088278D933197E9F76624BC9855
:10004000B898BA9AB99AB49AB09AC29AC198E4E0A8
:10005000F0E0A0E179D30F3609F009C0E0E0F0E06C
:10006000A3E774D3E2E0F0E0A5E770D312C082ED1D
:1000700090E0A3E78D939C938AE090E0A5E78D93B1
:100080009C93E4E0F0E0A0E1BB278FE68C937BE754
:100090004AD343D159D1C2988CE291E0E4D1C29ABB
:1000A0008CE291E0E0D10027A6E38C9184FB0EF472
:1000B00001E041E0041708F06EC0C298E2E0F0E011
:1000C000C3D1C29A0027A6E38C9180FB0EF401E015
:1000D00040E0041710F009F001C053C00027A6E368
:1000E0008C9184FB0EF401E041E0041708F048C055
:1000F000A3E70D911C914AE050E0040F151FA3E700
:100100000D931C93A3E70D911C910C3251E0150740
:1001100014F009F001C005C082ED90E0A3E78D93D3
:100120009C93A3E70D911C9148EC50E0041B150B28
:10013000A8E70D931C93A8E70D911C914AE050E0AD
:1001400036D1A8E74D935C9381E080937700A8E7D0
:100150004D915C91A7E70D9111270417150714F035
:1001600009F00EC0C29888EC90E07DD1C29A88EC6C
:1001700090E079D1A7E78C918F5F8C9308F4E7CF5B
:10018000A1CFE0E0F0E0A3E77BE7CFD2C298E1E0C7
:10019000F0E05AD1C29A0027A6E38C9180FB0EF4BE
:1001A00001E041E0041708F06AC0C298E2E0F0E024
:1001B0004BD1C29A0027A6E38C9184FB0EF401E098
:1001C00040E0041710F009F001C04FC00027A6E37B
:1001D0008C9180FB0EF401E041E0041708F044C06C
:1001E000A5E70D911C914AE050E0040F151FA5E70B
:1001F0000D931C93A5E70D911C91043650E0150753
:1002000014F009F001C005C08AE090E0A5E78D93E5
:100210009C93A5E78D919C91A8E78D939C93A8E76B
:100220000D911C914AE050E0C2D0A8E74D935C9339
:1002300081E080937700A8E74D915C91A7E70D914D
:1002400011270417150714F009F00EC0C29888ECA6
:1002500090E009D1C29A88EC90E005D1A7E78C9193
:100260008F5F8C9308F4E7CFA5CFE2E0F0E0A5E73D
:100270007BE75BD2C298E1E0F0E0E6D0C29AA3E768
:100280000D911C9141E050E0041B150BAAE70D9362
:100290001C93A3E70D911C91A5E74D915C91041B64
:1002A000150BACE70D931C9383E0E6E39CD1A0E62D
:1002B000E2E8F0E098E02DD2002762FA0EF401E0C7
:1002C00040E0041710F009F001C009C0C29888ECA2
:1002D00090E0C9D0C29A88EC90E0C5D01DC01DD076
:1002E00033D0A3E74D915C91A1E70D911C910417C8
:1002F000150714F009F001C002C0C298C19AACE71A
:100300004D915C91A1E70D911C91041715070CF418
:1003100001C002C0C29AC198C7CF83E0E6E3CCD047
:100320006CEC83E0E6E3BB27A6E121E02A93F0D062
:1003300064E483E0E6E3BB27A6E121E02A93E8D06A
:1003400080E293E090D0089583E0E6E3A0E6BED19A
:100350006EEB83E0E6E3BB27A6E121E02A93D8D049
:1003600083E0A8E6E6E329E02A93F0D0A9E69C9191
:10037000A8E68C91A1E78D939C93A1E70D911C9128
:100380004AE050E00FD0A1E70D931C93A1E70D9137
:100390001C9140E150E00BD0A1E74D935C93089590
:1003A000F894FFCF08D03DD000FC10D0089503D0C2
:1003B0001ED001F8F9CF0024E89457FF02C009D0FD
:1003C000689400F80BD010F80124089502D009D0E9
:1003D0000895509540954F5F5F4F0895E89417FF3B
:1003E0000895009510950F5F1F4F68940895352F5D
:1003F000242FE894452B11F468940895512F402F31
:100400000027112780E1440F551F001F111F021BF9
:10041000130B416018F4020F131F4E7F8A9599F752
:100420000895752F642F55274427FF93F1E1889491
:1004300005C010F4460F571F569547951795079519
:10044000FA95B9F7FF91089588EE93E00CD03197B3
:10045000D9F708953197F1F70895689462F80895EF
:10046000E89462F80895EF93FF93EE27E82BE92BC9
:1004700031F0EAEFF0E03197F1F70197D1F7FF9112
:10048000EF91089591E0882321F08894991F8A952F
:10049000E9F7892F90950895883018F011968850C3
:1004A000FBCF08950181082B018312811923128348
:1004B0000000000000000895D0DFFF27E3DFF2DF37
:1004C000EF93FF93E4E7F0E0C5DFFF91EF91182B86
:1004D000128309230183EF93FF93E3E1F0E0BADF96
:1004E000FF91EF911081182359F4EF93FF93E4E704
:1004F000F0E0B0DFFF91EF911081182309F0B0DF39
:10050000EF93FF93E4E7F0E0A5DFFF91EF9108950B
:10051000B9DFFF2729915D9148E0C4DF00000000AA
:100520000000579510F4182B1283EF93FF93EBE024
:10053000F0E090DFFF91EF91182B12830000000094
:1005400000004A9551F72A9531F708959BDFFF2760
:10055000299148E05527A6DF092301830000000008
:1005600000000000000000000000889410811823A3
:1005700009F008945795EF93FF93E8E0F0E06ADF05
:10058000FF91EF914A9539F75D932A9511F70895F8
:1005900089DF092301830000000000000000000043
:1005A00000000000E8941081182309F06894EF938C
:1005B000FF93E9E0F0E04EDFFF91EF91089572DFE5
:1005C00000000000000016F4182B1283EF93FF9335
:1005D000EBE0F0E03FDFFF91EF91182B128300007A
:1005E00000000000089533273093810030937E008F
:1005F00063DF0EF457C030917E0030FD53C0662794
:1006000060938000639560937F0021E050EF48E0A5
:1006100084DFBEDF31F9BCDF32F9632F66706630EC
:1006200009F440C0603019F031FB3FD024C0609124
:100630007F00709181006717A9F0B8F48F939F93A2
:10064000862F8A95A2E828DF1DDF7C9178236894A5
:10065000772329F4E89460917F00609380009F9154
:100660008F9109C0689421D006C0E8941ED0609193
:100670007F0060938000A3DF60917F0063956093AB
:100680007F00613409F0C5CF6091800060938100E4
:100690006623E89409F4689430F930937E00E89476
:1006A00062F80895689462F808958F939F93A2E882
:1006B00080917F008A95F0DEE5DE7C9116F4782B40
:1006C00001C079237C939F918F910895AF93BF933D
:1006D000EF93FF9338E0E2E8F0E00D9101933A9553
:1006E000E1F7FF91EF9130E43093810033273093AD
:1006F0007E007EDF38E0BF91AF91E2E8F0E00D913F
:100700004191041719F43A95D1F70895A6DE08959A
:1007100094E081918D939A95E1F70895E199FECF48
:10072000EEBB3196089591E001C092E07B3751F421
:100730007FB7F894F3DF8D918DBBE29AE19A9A9599
:10074000C9F77FBF7727089591E001C092E0E6DF07
:0C075000E09A8DB38D939A95D1F708952F
:00000001FF
